:020000040000FA
:100000007002040000000000FC100000FC10000062
:10001000FC100000FC100000FC100000FC100000B0
:10002000FC100000FC100000FC100000FC100000A0
:10003000FC100000FC100000FC100000FC10000090
:10004000FC1000005C090000FC100000FC10000027
:10005000FC100000FC100000FC100000FC10000070
:10006000FC100000FC100000FC100000FC10000060
:10007000FC100000FC100000FC100000FC10000050
:10008000FC100000FC100000FC100000FC10000040
:10009000FC100000FC100000D0060000FC10000066
:1000A000FC100000FC100000FC100000FC10000020
:1000B000FC100000FC100000FC100000FC10000010
:1000C000FC100000FC100000FC100000FC10000000
:1000D000FC100000FC100000FC100000FC100000F0
:1000E000FC100000FC100000FC100000FC100000E0
:1000F000FC100000FC100000FC100000FC100000D0
:10010000FC100000FC100000FC100000FC100000BF
:10011000FC100000FC100000FC100000FC100000AF
:10012000FC100000FC100000FC100000FC1000009F
:10013000FC100000FC100000FC100000FC1000008F
:10014000FC100000FC100000FC100000FC1000007F
:10015000FC100000FC100000FC100000FC1000006F
:10016000FC100000FC100000FC100000FC1000005F
:10017000FC100000FC100000FC100000FC1000004F
:10018000FC100000FC100000FC100000FC1000003F
:10019000FC100000FC100000FC100000FC1000002F
:1001A000FC100000FC100000FC100000FC1000001F
:1001B000FC100000FC100000FC100000FC1000000F
:1001C000FC100000FC100000FC100000FC100000FF
:1001D000FC100000FC100000FC100000FC100000EF
:1001E000FC100000FC100000FC100000FC100000DF
:1001F000FC100000FC100000FC100000FC100000CF
:10020000FFFFFF00FFFFFF00FC100000FC100000DC
:10021000FC100000FC100000FC100000FC100000AE
:10022000FC100000FC100000FC100000FC1000009E
:10023000FC100000FC100000FC100000FC1000008E
:10024000FC1000005C090000FC100000FC10000025
:10025000FC100000FC100000FC100000FC1000006E
:10026000FC100000FC100000FC100000FC1000005E
:10027000FC100000FC100000FC100000FC1000004E
:10028000FC100000FC100000FC100000FC1000003E
:10029000FC100000FC100000D0060000FC10000064
:1002A000FC100000FC100000FC100000FC1000001E
:1002B000FC100000FC100000FC100000FC1000000E
:1002C000FC100000FC100000FC100000FC100000FE
:1002D000FC100000FC100000FC100000FC100000EE
:1002E000FC100000FC100000FC100000FC100000DE
:1002F000FC100000FC100000FC100000FC100000CE
:10030000FC100000FC100000FC100000FC100000BD
:10031000FC100000FC100000FC100000FC100000AD
:10032000FC100000FC100000FC100000FC1000009D
:10033000FC100000FC100000FC100000FC1000008D
:10034000FC100000FC100000FC100000FC1000007D
:10035000FC100000FC100000FC100000FC1000006D
:10036000FC100000FC100000FC100000FC1000005D
:10037000FC100000FC100000FC100000FC1000004D
:10038000FC100000FC100000FC100000FC1000003D
:10039000FC100000FC100000FC100000FC1000002D
:1003A000FC100000FC100000FC100000FC1000001D
:1003B000FC100000FC100000FC100000FC1000000D
:1003C000FC100000FC100000FC100000FC100000FD
:1003D000FC100000FC100000FC100000FC100000ED
:1003E000FC100000FC100000FC100000FC100000DD
:1003F000FC100000FC100000FC100000FC100000CD
:1004000000000000000000000000000000000000EC
:1004100000000000000000000000000000000000DC
:10042000303200002C120000100E00000C0A0000F8
:100430002A280000260800002422000020060000D0
:10044000041E00001C1A000018160000142E0000E4
:10045000646600006046000044420000403E000028
:100460005E5C00005A3C000058560000543A000000
:1004700038520000504E00004C4A00004862000014
:100480000C4000000A3E00002A5E0000285C0000CC
:10049000265A0000083C00002458000022560000A4
:1004A00020540000063A0000043800001E520000EC
:1004B0001C5000001A4E0000184C0000164A0000A4
:1004C000144800002E620000306400003266000014
:1004D0002C60000012460000104400000E42000094
:1004E0004507A900F0012000403A8800CFE720002E
:1004F00000FF2000000188000000000081E0A8004B
:1005000000002000A00188004440A8000000EB008B
:100510003C0009000060FE000000E900FCFF3A001A
:1005200040802000F00CFC003B0309000018EB00A9
:10053000CC22EF00D422EF00C542A900C022EF0078
:10054000C822EF00D022EF00C622EF00CE22EF003B
:10055000D622EF00C002A800E004A9006E40A80067
:10056000820C0200000000000040880001E8AF009B
:1005700004A8A80001E8A90060012000500D88002F
:10058000C0002000300D8800E00D200060088800C9
:1005900011E1A80094E0A800F0FF270010088800EF
:1005A00005E1A8000060FE008460AE00FDFF37009A
:1005B0008460A9008A080200000000001208AE0052
:1005C00001003700F7FF37001228EF00E08120001C
:1005D000BC0CFC002E0309000018EB0000002800F2
:1005E000C04088000408A9000428A9000448A90004
:1005F00000AF2000F040880000B52000B044880023
:1006000000BB2000704888000003200000418800E3
:10061000C044880080488800F00F200050418800C6
:1006200010458800D0488800904C880050508800C1
:1006300010548800A00020000008E30001003600EC
:100640000028EF0000408000006001000D0037002E
:10065000260037006B0037009800370096003700FF
:10066000C9003700ED003700150137003D013700A4
:1006700073013700870137003408A800AC08A800D0
:100680002409A80000242000E0408800E028280079
:1006900060418800E051280020458800D07A280079
:1006A000E04888001000200030418800F0448800B5
:1006B000B04888004041880000458800C048880054
:1006C000A000200020418800E0448800A048880065
:1006D00000AF20008F00090030F0A000F1EAA9006F
:1006E00071EBA900F1EBA900B00137000021200057
:1006F000E040880000AF20009000FC008F0009005F
:1007000030F0A00000AF2000F040880000B52000CD
:10071000B044880000BB2000704888003408A8005E
:10072000AC08A8002409A80080012000004188002E
:10073000C044880080488800E02828006041880084
:10074000E051280020458800D07A2800E048880041
:100750001000200030418800F0448800B048880034
:100760004041880000458800C0488800A000200063
:1007700020418800E0448800A0488800F1EAA900F0
:1007800061EBA900D1EBA90000B22000304C880039
:1007900000B82000F04F880000BE2000B053880051
:1007A00080012000404C880000508800C053880021
:1007B000E0282800A04C8800E05128006050880004
:1007C000D07A28002054880010002000704C880047
:1007D00030508800F0538800804C880040508800DA
:1007E00000548800A0002000604C88002050880041
:1007F000E053880021EBA90091EBA90001ECA900CE
:100800006A01370000212000E0408800000020003D
:1008100010418800000C2000D044880000182000FF
:1008200090488800A0CE250060418800F0FF250098
:1008300020458800701C2600E04888001000200039
:1008400030418800F0448800B0488800404188006A
:1008500000458800C04888004000200020418800F2
:1008600040002000E044880040002000A0488800AC
:1008700000AF20008F00090030F0A000F1EAA900CD
:1008800051EBA900B1EBA9003428A800AC28A800BE
:100890002429A800100020008041880040458800DD
:1008A00000498800F00F20009041880050458800E2
:1008B000104988003D0137002409A8000428A80039
:1008C00000242000E0408800A05F20005041880004
:1008D00000C12000F040880000C72000B04488001C
:1008E00000CD2000704888000000200010418800E2
:1008F000D0448800904888000000210060418800B2
:10090000F0FF2F0020458800F0FF2F00E04888000E
:100910001000200030418800F00F2000F0448800D3
:1009200000022000B0488800A05F200040418800FD
:10093000000020000045880010002000C04888000A
:10094000100020002041880000002000E0448800C2
:1009500020002000A048880000C120008F0009006E
:1009600030F0A00011ECA90071ECA900D1ECA900B5
:100970002429A80010002000004988000000200061
:1009800010498800090137000428A80000602000F1
:100990005041880000C12000F040880000C72000BE
:1009A000B044880000CD200070488800000020007E
:1009B00010418800D044880090488800F0FF200053
:1009C00060418800F0FF2F0020458800F0FF2F00D5
:1009D000E04888001000200030418800F00F20001F
:1009E000F044880010002000B0488800006020001B
:1009F000404188000000200000458800C048880071
:100A0000400020002041880000C120002F00090084
:100A100030F0A00011ECA900E40037000024200011
:100A2000E0408800000020001041880000202000E5
:100A3000D04488000040200090488800F0FF2F003C
:100A40006041880020458800E048880010002000B0
:100A500030418800F0448800B04888004041880058
:100A600000458800C04888005000200020418800D0
:100A7000E0448800A048880000AF20008F000900F3
:100A800030F0A000F1EAA90051EBA900B1EBA900F8
:100A90003428A800AC28A8002429A80010002000B1
:100AA000804188004045880000498800C03F200000
:100AB000904188005045880010498800BB003700ED
:100AC0000428A800007720007057880000602000EC
:100AD0005041880000C12000F040880000C720007D
:100AE000B044880000CD200070488800F0FF2F003F
:100AF0006041880020458800E04888001000200000
:100B00003041880000002000F0448800F0032000FD
:100B1000B0488800A05F200040418800000020000D
:100B20000045880010002000C04888001000200008
:100B300020418800E044880000102000A048880080
:100B400000CD20002F00090030F0A0002429A800CB
:100B50001000200000498800000020001049880093
:100B6000920037000428A800A07920007057880060
:100B7000006020005041880000C12000F040880043
:100B800000C72000B044880000CD200070488800D5
:100B9000F0FF2F0060418800E0488800F0FF270048
:100BA0002045880000302000D0448800200020002C
:100BB0003041880010002000F0448800F00320003D
:100BC000B0488800A05F200040418800100020004D
:100BD0000045880010002000C04888000002200066
:100BE0002041880010002000E04488000010200010
:100BF000A048880000C120002E00090030F0A000AD
:100C000000C720002E00090030F0A00000CD200019
:100C10002F00090030F0A000AC28A8002429A8006B
:100C2000003020004045880050458800100020001A
:100C30000049880000002000104988005B00370050
:100C4000A07B200070578800F0FF270060418800DB
:100C500020458800E04888001000200030418800CE
:100C6000F0448800B0488800404188000045880072
:100C7000C04888000000200020418800E04488002F
:100C8000A048880000AF20008F00090030F0A000CD
:100C900046003700407D2000705788000428A800D7
:100CA00000242000E0408800A05F20005041880020
:100CB00000C12000F040880000C72000B044880038
:100CC00000CD2000704888000000200010418800FE
:100CD000D0448800904888000000200060418800CF
:100CE00020458800F0FF2F00E04888000002200027
:100CF000B048880010002000C04888002000200074
:100D0000A048880000CD20002F00090030F0A0008E
:100D1000D1ECA9002429A800100020000049880077
:100D2000000020001049880000C72000F10F2000BB
:100D30002F000900011878001C0037000060FE0039
:100D400040A7A90005E1A90094E0A90084E0AE0055
:100D5000FEFF370011E1A90084E0A9009780A900F7
:100D60008780A900C0A2EF00C8A2EF00D0A2EF00C8
:100D7000C202AE00FEFF37000000EB0018000900C1
:100D8000000000000000E900FCFF3A008660A900B6
:100D90006240A8009660A8000040FE000000FE002F
:100DA0008780A9001248A800004006000060FE00ED
:100DB00040A7A80094E0A8008460AE00FEFF3700C2
:100DC0008460A9008A080200000000001228AF0019
:100DD000DAFF37001248AE000E0037001248A900B3
:100DE0000028EC0094E0A9000060FE0084E0AE0062
:100DF000FDFF37000040800004A8AF0000F0A00015
:100E00005C0C0200000000000060FE0040A7A9008A
:100E1000EEFD3700C04080001A28B400E6FF39001C
:100E2000EE0AE2000200320070578000000001006C
:100E30000408A800E1812000CC08020000000000A6
:100E400061892000CC08020000000000E190200031
:100E5000CC080200000000008609E2000900320010
:100E600061982000CC08020000000000E19F2000F3
:100E7000CC0802000000000061A72000CC0802009E
:100E8000000000000428AF004C0702000000000032
:100E90000408A900C8FF370003C1200007AF2000E5
:100EA000E9B42000F0FF2300130278000402600080
:100EB000833290008502600003A390000603600067
:100EC000EE070200000000000938E10003003200D4
:100ED0008381E8008783E800F2FF37000000060006
:100EE00003CD200009D320008C0C0200000000007C
:100EF00001F02F000100E1000A0039001304E000B6
:100F000008003A0013F0A100F10F2000010060007A
:100F10006600B80080219F008C0C020000000000D9
:100F200080619F008381E8000918E100EEFF3A002C
:100F30000000060003CD200009D320008C0C020025
:100F400000000000010020000100E1000500390060
:100F50001304E00003003A008049780013E0A00089
:100F600013F0A1008381E8000918E100F3FF3A00C3
:100F70000000060003AF200009C120008C0C020015
:100F8000000000001304E00003003A0080497800EC
:100F900013E0A00013F0A1008381E8000918E1002C
:100FA000F6FF3A000000060003CD200009D3200020
:100FB0001304E00005003A008C0C02000000000061
:100FC000F15F20000100600080219F008381E80024
:100FD0000918E100F6FF3A00000006000500E000F5
:100FE00004003A00860B78008633980086A39800A8
:100FF00000000600A47388004820DE00907388007B
:101000004800DD00742EB5000010200005005000DF
:101010000600B8004800DE00B0738800A0738000AE
:101020000500B8004800DE000000EA000010B00033
:101030000600B8004800DE00C0738800A07380007E
:101040000000EA000010B0000500B8004800DE0013
:101050000000EA000010B0000600B8004800DE0002
:10106000D073880090738000006001000500370095
:101070000A0037000F00370014003700190037004E
:101080001E003700860B7800D073800080339800F4
:10109000B073800080A3980000000600C073800039
:1010A000800B780086339800B073800080A398008E
:1010B00000000600B0738000800B78008633980033
:1010C000D073800080A3980000000600B0738000F9
:1010D000800B7800C07380008033980086A398004E
:1010E00000000600D0738000800B7800B073800091
:1010F0008033980086A3980000000600860B7800D5
:10110000B073800080339800C073800080A3980083
:1011100000000600101680000000A30014A8D600EE
:101120002181200098080200000000000000060055
:101130001100A70008003700F0FF2F0011019000F8
:101140000201600003003A001100A000A00F20007F
:10115000A000980000000600F0FF2F001101900091
:10116000020160000001690003003A001100A100C3
:101170001120A00000000600648140001209E9006F
:1011800001003200000006001110A000A00F200096
:10119000A00098000000060071009000F08140005F
:1011A0009309400001003100000006006480400007
:1011B0001000E000020032001008E9000000060004
:1011C00081049000110090000000E9000000D000B0
:1011D0008085440041069000D106900031049000C3
:1011E0006107900088035700310B90000600A700AC
:1011F0000200370062854400010037000B057800CB
:10120000F8824000F0FF23001900600019F0A600EA
:1012100003003700950AE9001B003A0019F0A1000D
:1012200019E0A7000D0037000040E7001AF0A10008
:101230000C0040000E00E100130039000E007800A1
:1012400019E0A2000610A6000F00370019F0A00058
:1012500091099000830A78000B0037000038E700FE
:101260001AF0A1000D005000070031000000EB0053
:1012700019E0A2000610A6000300370019F0A00034
:10128000A1099000830A780003002C00998C61006A
:10129000990C70000B48E700000006008582E8000A
:1012A0008984E8000A85E8000B50E600D5FF370086
:1012B00001059000D3FF370000A0FE00849FBE0010
:1012C00034ADBF003800320040C02100200D88003E
:1012D00070738000817380009269800022168800FC
:1012E00060168800A11688008069800000600100F7
:1012F000060037000C0037001200370018003700D6
:101300001E00370024003700302DEF00E1D9200007
:10131000E2E6200000102000906988003A0A0200EE
:10132000000000004D00370061E02000E2E62000F0
:1013300000002000906988003A0A020000000000C6
:1013400046003700A1D62000E2E620004010200031
:10135000906988003A0A0200000000003F00370050
:1013600021DD2000E2E62000400020009069880096
:101370003A0A02000000000038003700A1E3200014
:10138000E2E6200080102000906988003A0A0200FE
:10139000000000003100370034ADEC00F00F2000F9
:1013A000340DE300230036000408AF001F003700AF
:1013B0001CA8BF0002003A0000212000E040880085
:1013C00000002000900188000000EB00E540800054
:1013D00001AF200004B5200062D320003540BA00E0
:1013E000313178000408E100FCFF3A00E54080005C
:1013F00001B5200004BB2000E2D920003540BA002E
:10140000313178000408E100FCFF3A00E54080003B
:1014100001BB200004C1200062E020003540BA007A
:10142000313178000408E100FCFF3A00342DEF0070
:10143000342DEC00C3A52800340DD40063007800DF
:10144000400D880061D32000E2E6200080002000EB
:10145000906988003A0A020000000000302DEC007C
:101460000060FE004F02BE000080FE0084E0A90084
:1014700000400600A36980000400280004097800E9
:10148000310078000304E1001289D300FCFF390029
:101490000281E8000420200004097800310078006F
:1014A0000304E1001289D300FCFF390005000900A4
:1014B0001209D1000000060017000000170000000C
:1014C00017000000170000001700000017000000C0
:1014D00017000000170000001800000019000000AD
:1014E0001A0000001A0000001B0000001C00000091
:1014F0001D0000001E0000001E0000001F00000074
:101500002000000021000000220000002200000056
:101510002300000024000000250000002600000039
:10152000260000002700000028000000290000001D
:101530002A0000002A0000002B0000002C00000000
:101540002D0000002E0000002E0000002F000000E3
:1015500030000000310000003200000032000000C6
:1015600033000000340000003500000036000000A9
:10157000360000003700000038000000390000008D
:10158000390000003A0000003B0000003C00000071
:101590003D0000003D0000003E0000003F00000054
:1015A0004000000041000000410000004200000037
:1015B000430000004400000045000000450000001A
:1015C00046000000470000004800000049000000FD
:1015D000490000004A0000004B0000004C000000E1
:1015E0004D0000004D0000004E0000004F000000C4
:1015F00050000000510000005100000052000000A7
:101600005300000054000000550000005500000089
:10161000560000005700000058000000590000006C
:10162000590000005A0000005B0000005C00000050
:101630005C0000005D0000005E0000005F00000034
:101640006000000060000000610000006200000017
:1016500063000000640000006400000065000000FA
:1016600066000000670000006800000068000000DD
:10167000690000006A0000006B0000006C000000C0
:101680006C0000006D0000006E0000006F000000A4
:101690007000000070000000710000007200000087
:1016A000730000007400000074000000750000006A
:1016B000760000007700000078000000780000004D
:1016C000790000007A0000007B0000007B00000031
:1016D0007C0000007D0000007E0000007F00000014
:1016E0007F000000800000008100000082000000F8
:1016F00083000000830000008400000085000000DB
:1017000086000000870000008700000088000000BD
:10171000890000008A0000008B0000008B000000A0
:101720008C0000008D0000008E0000008F00000083
:101730008F00000090000000910000009200000067
:10174000930000009300000094000000950000004A
:10175000960000009700000097000000980000002D
:10176000990000009A0000009B0000009B00000010
:101770009C0000009D0000009E0000009E000000F4
:101780009F000000A0000000A1000000A2000000D7
:10179000A2000000A3000000A4000000A5000000BB
:1017A000A6000000A6000000A7000000A80000009E
:1017B000A9000000AA000000AA000000AB00000081
:1017C000AC000000AD000000AE000000AE00000064
:1017D000AF000000B0000000B1000000B200000047
:1017E000B2000000B3000000B4000000B50000002B
:1017F000B6000000B6000000B7000000B80000000E
:10180000B9000000BA000000BA000000BB000000F0
:10181000BC000000BD000000BD000000BE000000D4
:10182000BF000000C0000000C1000000C1000000B7
:10183000C2000000C3000000C4000000C50000009A
:10184000C5000000C6000000C7000000C80000007E
:10185000C9000000C9000000CA000000CB00000061
:10186000CC000000CD000000CD000000CE00000044
:10187000CF000000D0000000D1000000D100000027
:10188000D2000000D3000000D4000000D50000000A
:10189000D5000000D6000000D7000000D8000000EE
:1018A000D9000000D9000000DA000000DB000000D1
:1018B000DC000000DD000000F1072000910188003D
:1018C00001E02F008008BB006027EF0061C7A8007F
:1018D0006047A8000700FC0051052000313B88004C
:1018E000A10A2000313B880061E7A8000000000049
:1018F000000000000060FE0061E7AF00FDFF370060
:1019000000000600F00720009001880000E02F0092
:101910001000BA000000060000402B004200A900A1
:1019200002A8D7004200AF0002A8B6004220AF00D4
:101930000228EC0010408000000006000000FE00BD
:10194000000800007C06000002000000000000000B
:101950000000000000000000000000000000000087
:101960000000000000000000000000000000000077
:101970000000000000000000000000000000000067
:101980000000000000000000000000000000000057
:1021F00000000000000000000040DA000000FE00C7
:10220000FFFFFF00FFFFFF00FFFFFF00FFFFFF00DA
:10221000FFFFFF00FFFFFF00FFFFFF00FFFFFF00CA
:10222000FFFFFF00FFFFFF00FFFFFF00FFFFFF00BA
:10223000FFFFFF00FFFFFF00FFFFFF00FFFFFF00AA
:0200000400FFFB
:0200000401F009
:100000000F000000000000000300000001000000DD
:10001000CB000000C0000000DF00000083000000F3
:0400200014000000C8
:00000001FF
